:100000000C9445000C9462000C9462000C94620005
:100010000C9462000C9462000C9462000C946200D8
:100020000C9462000C9452040C9462000C946200D4
:100030000C9462000C942D050C9462000C946200E8
:100040000C9462000C9462000C9462000C946400A6
:100050000C94620005A84CCDB2D44EB93836A90232
:100060000C50B9918688083CA6AAAA2ABE000000B6
:10007000803F45464765666700202B2D2E30313284
:100080003334353637383968000011241FBECFE5C8
:10009000D8E0DEBFCDBF10E0A0E6B0E0EAE3F7E2D3
:1000A00002C005900D92A837B107D9F721E0A8E763
:1000B000B0E001C01D92A736B207E1F70E94220608
:1000C0000C949B130C9400001F920F920FB60F928A
:1000D00011242F933F934F935F936F937F938F934D
:1000E0009F93AF93BF93EF93FF9381B1887F803845
:1000F00081F040F4803609F0BFC385EC86BF1092D2
:10010000E800BFC3883A09F4B7C1883B09F4B4C119
:10011000B3C38091E8008A3209F449C108F047C0AE
:10012000803209F402C138F5843009F4C1C060F4AA
:10013000813009F4FAC008F4A6C0823009F4ACC0DA
:10014000833009F4F2C090C3863009F4BDC008F4CE
:10015000ECC0873009F4E9C0883009F085C383B169
:100160002091A60090E0922B9093E0008093DF0016
:100170001092D30071C3853209F4CAC060F4823290
:1001800009F4D3C008F4ACC0833209F4B6C0843299
:1001900009F4CBC069C3873209F4CBC008F4C5C0E9
:1001A000883209F4FFC0893209F401C15DC3843586
:1001B00009F414C1E8F58F3209F4C8C060F48C3238
:1001C00009F4F0C008F4C2C08D3209F4F0C08E32D8
:1001D00009F4EDC049C3813509F4E9C020F4803544
:1001E00009F4E0C041C3823509F4E1C0833509F068
:1001F0003BC323B18091A2009091A300A091A400E1
:10020000B091A500BA2FA92F982F8827822B809311
:10021000A2009093A300A093A400B093A5008093A4
:10022000E9009093EA00A093EB00B093EC0014C3B4
:10023000813909F40EC178F4863509F4D4C008F484
:10024000D2C0873509F4E6C0803909F00DC383B107
:100250008093D20001C3843909F403C150F4823978
:1002600009F4FBC0833909F0FFC283B18093CF004A
:10027000F3C2853909F4F9C08F3F09F0F5C283B1A3
:100280008093E700F1C283B18093E8008091E80099
:1002900081508093E800E0C283B12091A60090E0F5
:1002A000922B9093E6008093E5001092D600D4C282
:1002B00083B12091A60090E0922B9093E40080936C
:1002C000E3001092D500C8C283B12091A60090E04F
:1002D000922B9093E2008093E1001092D400BCC274
:1002E00083B12091A60090E0922B9093CE00809352
:1002F000CD0081E08093D600AFC283B12091A600EB
:1003000090E0922B9093CC008093CB0081E047C08B
:1003100083B12091A60090E0922B9093CA00809325
:10032000C90081E08093D40097C283B18093A60076
:1003300093C283B12091A60090E0922B9093C800C5
:100340008093C70081E08093D30086C223B180915F
:10035000A2009091A300A091A400B091A5006627EF
:10036000782F892F9A2F622B6093A2007093A3009D
:100370008093A4009093A50023E33BE542E855E475
:100380000E9450100E94300F7093CE006093CD00F9
:100390007093CC006093CB0081E08093D600809373
:1003A000D5005AC283B190E0A0E0B0E00EC023B106
:1003B0008091A2009091A300A091A400B091A5000B
:1003C000BA2FA92F982F8827822B8093A200909371
:1003D000A300A093A400B093A5003EC283B190E017
:1003E000A0E0B0E00EC023B180919E0090919F00EC
:1003F000A091A000B091A100BA2FA92F982F882713
:10040000822B80939E0090939F00A093A000B093B6
:10041000A10022C223B180919E0090919F00A091E3
:10042000A000B091A100BA2FA92F982F8827822B66
:1004300080939E0090939F00A093A000B093A10092
:100440008093ED009093EE00A093EF00B093F00046
:100450000FC083B18093D100FFC183B18093D000DE
:10046000FBC183B18093A80003C083B18093A70030
:1004700081E08093F100F0C18091E800853309F4B8
:1004800047C108F06BC0803209F415C180F5813195
:1004900009F40EC1C0F4863009F4F2C048F4823089
:1004A00009F4EBC0843009F0DEC188B599B5E9C024
:1004B000883009F4E8C0803109F0D5C18091DD00B1
:1004C0009091DE00F0C0843109F4E4C038F4823148
:1004D00009F4DBC0833109F4EBC0C5C1863109F4EE
:1004E000DEC008F4E5C0873109F4E2C0BCC1863241
:1004F00009F4F5C0D0F4833209F4E7C058F481322E
:1005000009F4DEC0823209F0AEC18091CB00909137
:10051000CC0007C1843209F4DDC0853209F0A3C1E3
:100520008091C9009091CA00ACC0813309F4E1C048
:1005300058F4873209F4D8C0803309F094C180910F
:10054000C4009091C500EDC0833309F4D7C008F012
:10055000DAC08091C2009091C300E3C0823409F4F4
:1005600022C108F043C08B3309F4F7C0F0F488339C
:1005700009F4D9C058F4863309F4CFC0873309F0A1
:1005800072C18091BE009091BF007BC0893309F495
:10059000DBC08A3309F067C18091A2009091A3006B
:1005A000A091A400B091A5003BC18E3309F4E9C02D
:1005B00078F48C3309F4D4C08D3309F054C18091A0
:1005C0009E0090919F00A091A000B091A10024C135
:1005D000803409F4DFC008F428C18091BA009091FA
:1005E000BB00A091BC00B091BD0016C1883409F4D5
:1005F000FEC010F5853409F4E8C078F4833409F4BA
:10060000DBC0843409F02FC18091B6009091B7000F
:10061000A091B800B091B900F2C0863409F4DEC0F0
:10062000873409F020C18091B6009091B700A09165
:10063000B800B091B90025C08B3409F4F6C078F445
:10064000893409F4E1C08A3409F00DC18091B20007
:100650009091B300A091B400B091B500E1C0813A8F
:1006600009F4ECC0823A09F4F9C0803A09F0FBC001
:1006700084B78F7083B914BEEFC08AB59BB501C033
:1006800083B583B9E9C08CB7FCCF8091DB00909132
:10069000DC0009C08091D9009091DA0004C08091FB
:1006A000D7009091D80090939D0080939C0039C012
:1006B00080919C00E6CF8091CD009091CE0031C01A
:1006C0008091CD009091CE00DCCF8091CB009091B5
:1006D000CC00D7CF8091C9009091CA0022C08091F0
:1006E000C7009091C8001DC08091C7009091C800BC
:1006F000C8CF8091C4009091C500C3CF8091C20043
:100700009091C300BECF8091C0009091C10009C0FC
:100710008091C0009091C100B4CF8091BE009091B3
:10072000BF0093B999C08091AE009091AF00A091A5
:10073000B000B091B1008093A2009093A300A09369
:10074000A400B093A5005BC08091A2009091A3008B
:10075000A091A400B091A5005FC08091A20091CFAC
:100760008091AA009091AB00A091AC00B091AD0037
:1007700080939E0090939F00A093A000B093A1004F
:100780003EC080919E0090919F00A091A000B091EA
:10079000A10046C08091BA009091BB00A091BC001E
:1007A000B091BD002CC08091BA009091BB00A09187
:1007B000BC00B091BD0034C08091BA009091BB00E4
:1007C000A091BC00B091BD005CCF8091B60090912B
:1007D000B700A091B800B091B9001EC08091B600DA
:1007E0009091B700A091B800B091B90019C0809164
:1007F000B2009091B300A091B400B091B5008B2FDE
:100800009927AA27BB273DCF8091B2009091B300D2
:10081000A091B400B091B500CD01AA27BB2731CF7C
:10082000892F9A2FAB2FBB272CCF8091B2009091AC
:10083000B300A091B400B091B50023CF80B326B32C
:10084000807490E033E0959587953A95E1F72770AD
:10085000282B20952F7023B985EC07C08091A90023
:1008600083B985EC86BF13B885E886BF8091E80020
:100870008F5F8093E80005C086B78B7E86BF85ECCE
:1008800086BFFF91EF91BF91AF919F918F917F9123
:100890006F915F914F913F912F910F900FBE0F90ED
:1008A0001F9018951F920F920FB60F9211242F933D
:1008B0003F934F935F938F939F9399B390FD02C0A3
:1008C00080E001C083E091FF02C091E08927209180
:1008D0009B00281B20FF1FC080939B008091D200AB
:1008E000422F4270882349F08091DD009091DE0014
:1008F000242F30E02150310908C08091DD00909113
:10090000DE0021E030E0241B3109820F931F909319
:10091000DE008093DD0099B392959F7090FD02C038
:1009200080E001C083E091FF02C091E0892720911F
:100930009A00281B20FF1FC080939A008091D1004D
:100940002270882359F08091DB009091DC0041E017
:1009500050E0421B5109840F951F09C08091DB00B4
:100960009091DC0030E021503109820F931F909369
:10097000DC008093DB0099B39695969590FD02C0BC
:1009800080E001C083E091FF02C091E089272091BF
:100990009900281B20FF1FC0809399008091D000F0
:1009A0002270882359F08091D9009091DA0041E0BB
:1009B00050E0421B5109840F951F09C08091D90056
:1009C0009091DA0030E021503109820F931F90930B
:1009D000DA008093D90099B3929596959695937085
:1009E00090FD02C080E001C083E0927011F091E0C0
:1009F000892720919800281B20FF1FC08093980012
:100A00008091CF00422F4270882349F08091D70017
:100A10009091D800242F30E02150310908C08091F6
:100A2000D7009091D80021E030E0241B3109820FDB
:100A3000931F9093D8008093D7008091C6008F5F5A
:100A40008093C6009F918F915F914F913F912F911D
:100A50000F900FBE0F901F9018951F920F920FB618
:100A60000F9211248F939F93EF93FF935F9B16C078
:100A7000E091F400F091F5008CB1808381E0E935DC
:100A8000F80730F43196F093F500E093F40006C0D7
:100A900086EF90E09093F5008093F400FF91EF9142
:100AA0009F918F910F900FBE0F901F9018959C01F2
:100AB0008AB188618AB9579A80B5866080BD40E066
:100AC00050E084E0220F331F441F551F8A95D1F751
:100AD00060E079E08DE390E00E94FD10DA01C90149
:100AE0000197A109B109892F9A2FAB2FBB27A7FD29
:100AF000BA9580BD215029B986EF90E09093F3001C
:100B00008093F2009093F5008093F40008955D9B2C
:100B1000FECFFC0180818CB90895CF93DF931F92A3
:100B2000CDB7DEB78983CE0101960E94870580E0AC
:100B300090E00F90DF91CF910895CF93DF93EC0178
:100B4000CE012196FC012081222319F00E94870505
:100B5000F7CFDF91CF9108955F9BFECF8CB190E0EE
:100B600008950C94AC0561EB75E08DE895E00C946C
:100B70004911CF93DF93FC01E253FF4FA081B18174
:100B8000EC01C453DF4F28813981A217B307A1F0CC
:100B90005D9B12C02C912CB920813181AC01455351
:100BA0005F4F2417350718F42F5F3F4F03C09C0198
:100BB00028593F4F31832083E091F200F091F300F8
:100BC0002091F4003091F5002E173F07C1F1DC01B0
:100BD000AC59BF4FCD91DC911197208128836D9145
:100BE0007C9111979C012B523F4FE9013881EB0119
:100BF0002881321307C09C012C523F4FE9014881E4
:100C00004F5F48839C012D593F4F6217730728F4AB
:100C1000EB012196CD93DC9302C08D939C93D1E0A0
:100C2000E935FD0730F43196F093F300E093F200DC
:100C300006C086EF90E09093F3008093F200DF917E
:100C4000CF910895CF93DF93CDB7DEB76E970FB6F0
:100C5000F894DEBF0FBECDBF88E087BB8CEF84BBAE
:100C60008CEB81BB87E088BB80E482BB1092E700FD
:100C700080E895E20E9457050E94B30580E582B99D
:100C800086B78B7E86BF85EC86BF81EF8FBD89E0FE
:100C90008EBD1BBC1ABC19BC18BC89E785BD13BC32
:100CA00083BF1CBE8EE690E00E94C61185B78F7888
:100CB00085BF84E089BF789474E6272E312C80911B
:100CC000E8008F3F41F48091E700853A21F4F894E1
:100CD000E0E0F8E109958091F100882309F407C16B
:100CE000F8948090E9009090EA00A090EB00B0901A
:100CF000EC006091ED007091EE008091EF0090911A
:100D0000F0001092F10078942BED3FE049E450E4BC
:100D10000E94501025E236E041E85EE30E94501048
:100D200020E030E040E05FE30E945010A501940114
:100D30000E945D0E6B017C01A5019401C501B40107
:100D40000E945D0EA70196010E945C0E23E33BE525
:100D500042E855E40E9450104B015C0123E33BE55F
:100D600042E855E4C701B6010E9450106B017C01B6
:100D700020E030E0A901C501B4010E944C10181612
:100D8000ECF48091A7008823C9F08091A70091011D
:100D9000281B3109B901882777FD8095982F0E947B
:100DA000630F9B01AC01C501B4010E94501020E00B
:100DB00030E048EC52E40E94C80E02C0C501B40104
:100DC0000E94300F7093CE006093CD0020E030E0A1
:100DD000A901C501B4010E94C10E87FF1DC0809109
:100DE000A8008823C9F08091A800A101481B5109DF
:100DF000BA01882777FD8095982F0E94630F9B0189
:100E0000AC01C501B4010E94501020E030E048EC74
:100E100052E40E94C80E02C0C501B4010E94300F06
:100E20007093CC006093CB0020E030E0A901C701B3
:100E3000B6010E94C10E87FF1CC08091A8008823C4
:100E4000C1F08091A800B101681B7109882777FD66
:100E50008095982F0E94630F9B01AC01C701B601DA
:100E60000E94501020E030E048EC52E40E94C80E8E
:100E700002C0C701B6010E94300F7093CA00609390
:100E8000C90020E030E0A901C701B6010E944C1062
:100E90001816E4F48091A7008823C1F08091A70080
:100EA000B101681B7109882777FD8095982F0E94F2
:100EB000630F9B01AC01C701B6010E94501020E0F6
:100EC00030E048EC52E40E94C80E02C0C701B601EF
:100ED0000E94300F7093C8006093C70051E0509398
:100EE000D6005093D5005093D4005093D3008091F6
:100EF000C6008C3908F48BC51092C600F894809116
:100F0000DD009091DE009A838983E091DB00F0910F
:100F1000DC00FC83EB832091D9003091DA003E8322
:100F20002D834091D7005091D80058874F837894F3
:100F30008091960090919700A980BA80A81AB90A6A
:100F400080919400909195008F01081B190B80915E
:100F50009200909193007901E81AF90A809190002B
:100F6000909191006A01C81AD90AB501882777FDC6
:100F70008095982F0E94630F2AE037ED43E25CE3EF
:100F80000E94C80E0E94300F69877A878B879C87E2
:100F9000B801882777FD8095982F0E94630F2AE07B
:100FA00037ED43E25CE30E94C80E0E94300F6D876C
:100FB0007E878F87988BB701882777FD8095982F3C
:100FC0000E94630F2AE037ED43E25CE30E94C80E03
:100FD0000E94300F698B7A8B8B8B9C8BB601882794
:100FE00077FD8095982F0E94630F2AE037ED43E24A
:100FF0005CE30E94C80E0E94300F6D8B7E8B8F8B3E
:10100000988FB501600F711F882777FD8095982F05
:101010000E94630F23E33BE542E056E40E94C80EC2
:101020004B015C01B7016C0D7D1D882777FD809514
:10103000982F0E94630F23E33BE542E056E40E94B1
:10104000C80E2B013C01C090B200D090B300E090DC
:10105000B400F090B500A50194010E945C0E25E259
:1010600036E041E85EE30E94C80E9B01AC01C70177
:10107000B6010E945D0E6B017C012BED3FE049EC57
:1010800050E40E944C1018164CF42BED3FE049EC54
:1010900050E4C701B6010E945C0E12C02BED3FE088
:1010A00049EC50ECC701B6010E94C10E87FF0AC08F
:1010B0002BED3FE049EC50E4C701B6010E945D0E04
:1010C0006B017C01A3019201C501B4010E945D0E78
:1010D00020E030E040E05FE30E9450104B015C01F3
:1010E0004090BA005090BB006090BC007090BD0072
:1010F000C701B6010E94C50EA50194010E945010BF
:101100009B01AC01C301B2010E945D0E698F7A8F11
:101110008B8F9C8F4090B6005090B7006090B800C5
:101120007090B900C701B6010E94B310A5019401E7
:101130000E9450109B01AC01C301B2010E945D0EE0
:101140002B013C010D851E8589859A85080F191F85
:1011500017FF02C00F5F1F4F159507954D895E89D8
:10116000E989FA894E0F5F1F57FF02C04F5F5F4F3B
:101170009A01359527953E8F2D8FB901600F711F0C
:10118000882777FD8095982F0E94630F23E33BE526
:1011900042E056E40E94C80E4B015C016D8D7E8DCD
:1011A000601B710B882777FD8095982F0E94630F35
:1011B00027EB36E64EE455E40E94C80EF894C09240
:1011C000B200D092B300E092B400F092B500298D45
:1011D0003A8D4B8D5C8D2093BA003093BB004093C9
:1011E000BC005093BD004092B6005092B700609290
:1011F000B8007092B90049855A855093C500409354
:10120000C400ED85FE85F093C300E093C2002989F8
:101210003A893093C1002093C0004D895E89509374
:10122000BF004093BE008092AE009092AF00A092AB
:10123000B000B092B1006093AA007093AB008093AD
:10124000AC009093AD00789489819A819093970037
:1012500080939600EB81FC81F0939500E0939400DD
:101260002D813E8130939300209392004F815885C9
:1012700050939100409390008091D600813009F006
:10128000ABC08091CD009091CE00892B89F4109253
:10129000E6001092E50010928F0010928E001092DE
:1012A0008A0010928B0010928C0010928D0094C0D6
:1012B0000091CD001091CE008091C4009091C500A6
:1012C000081B190B2801662457FC6094762CC090EB
:1012D0008A00D0908B00E0908C00F0908D00C40CC0
:1012E000D51CE61CF71CC0928A00D0928B00E092BD
:1012F0008C00F0928D008091E5009091E600BC0199
:10130000882777FD8095982F0E94630F4B015C0121
:10131000C301B2010E94630F2CEB34E743E15CE3AD
:101320000E9450102B013C01C701B6010E94630FBF
:101330002BE631ED46E05AE30E9450109B01AC01D0
:10134000C301B2010E945D0E6B017C0180918E0091
:1013500090918F00F801E81BF90BBF01882777FDFA
:101360008095982F0E94630F2CE234ED4AE15DE3F3
:101370000E9450109B01AC01C701B6010E945D0E96
:101380009B01AC01C501B4010E945D0E0E94300FAB
:101390007093E6006093E50010938F0000938E0039
:1013A0008091E5009091E6008F3F910541F03CF07F
:1013B0002FEF30E03093E6002093E5000DC08091E0
:1013C000E5009091E60081309F4F34F441E05FEFFB
:1013D0005093E6004093E5008091D500813009F0FC
:1013E000ABC08091CB009091CC00892B89F41092F6
:1013F000E4001092E300109289001092880010928D
:10140000840010928500109286001092870094C08C
:101410000091CB001091CC008091C2009091C3004C
:10142000081B190B2801662457FC6094762CC09089
:101430008400D0908500E0908600F0908700C40C76
:10144000D51CE61CF71CC0928400D0928500E09267
:101450008600F09287008091E3009091E400BC0147
:10146000882777FD8095982F0E94630F4B015C01C0
:10147000C301B2010E94630F2CEB34E743E15CE34C
:101480000E9450102B013C01C701B6010E94630F5E
:101490002BE631ED46E05AE30E9450109B01AC016F
:1014A000C301B2010E945D0E6B017C018091880036
:1014B00090918900F801E81BF90BBF01882777FD9F
:1014C0008095982F0E94630F2CE234ED4AE15DE392
:1014D0000E9450109B01AC01C701B6010E945D0E35
:1014E0009B01AC01C501B4010E945D0E0E94300F4A
:1014F0007093E4006093E3001093890000938800E8
:101500008091E3009091E4008F3F910541F03CF021
:101510002FEF30E03093E4002093E3000DC0809182
:10152000E3009091E40081309F4F34F441E05FEF9D
:101530005093E4004093E3008091D400813009F09F
:10154000ABC08091C9009091CA00892B89F4109298
:10155000E2001092E100109283001092820010923B
:101560007E0010927F00109280001092810094C043
:101570000091C9001091CA008091C0009091C100F3
:10158000081B190B2801662457FC6094762CC09028
:101590007E00D0907F00E0908000F0908100C40C2D
:1015A000D51CE61CF71CC0927E00D0927F00E09212
:1015B0008000F09281008091E1009091E200BC01F6
:1015C000882777FD8095982F0E94630F4B015C015F
:1015D000C301B2010E94630F2CEB34E743E15CE3EB
:1015E0000E9450102B013C01C701B6010E94630FFD
:1015F0002BE631ED46E05AE30E9450109B01AC010E
:10160000C301B2010E945D0E6B017C0180918200DA
:1016100090918300F801E81BF90BBF01882777FD43
:101620008095982F0E94630F2CE234ED4AE15DE330
:101630000E9450109B01AC01C701B6010E945D0ED3
:101640009B01AC01C501B4010E945D0E0E94300FE8
:101650007093E2006093E100109383000093820096
:101660008091E1009091E2008F3F910541F03CF0C4
:101670002FEF30E03093E2002093E1000DC0809125
:10168000E1009091E20081309F4F34F441E05FEF40
:101690005093E2004093E1008091D300813009F043
:1016A000ABC08091C7009091C800892B89F410923B
:1016B000E0001092DF0010927D0010927C001092EA
:1016C00078001092790010927A0010927B0094C0FA
:1016D0000091C7001091C8008091BE009091BF009A
:1016E000081B190B2801662457FC6094762CC090C7
:1016F0007800D0907900E0907A00F0907B00C40CE4
:10170000D51CE61CF71CC0927800D0927900E092BC
:101710007A00F0927B008091DF009091E000BC01A4
:10172000882777FD8095982F0E94630F4B015C01FD
:10173000C301B2010E94630F2CEB34E743E15CE389
:101740000E9450102B013C01C701B6010E94630F9B
:101750002BE631ED46E05AE30E9450109B01AC01AC
:10176000C301B2010E945D0E6B017C0180917C007F
:1017700090917D00F801E81BF90BBF01882777FDE8
:101780008095982F0E94630F2CE234ED4AE15DE3CF
:101790000E9450109B01AC01C701B6010E945D0E72
:1017A0009B01AC01C501B4010E945D0E0E94300F87
:1017B0007093E0006093DF0010937D0000937C0045
:1017C0008091DF009091E0008F3F910541F03CF067
:1017D0002FEF30E03093E0002093DF000DC08091C8
:1017E000DF009091E00081309F4F34F441E05FEFE3
:1017F0005093E0004093DF008091E5009091E60077
:10180000209166003091670028173907B9F180915F
:10181000E5009091E600892B19F485B38C6017C020
:101820008091D200811107C08091E5009091E6007F
:101830001816190654F08091D200882351F0809137
:10184000E5009091E60097FF04C085B3837F85BBD8
:1018500002C0AA98AB9A8091E5009091E60090931F
:101860006700809366008091E5009091E60097FF05
:1018700003C09195819591099BBD8ABD8091E3003C
:101880009091E40020916400309165002817390799
:10189000B9F18091E3009091E400892B19F485B3AC
:1018A000806317C08091D100811107C08091E3004F
:1018B0009091E4001816190654F08091D100882305
:1018C00051F08091E3009091E40097FF04C085B34C
:1018D0008F7C85BB02C0AC98AD9A8091E30090915B
:1018E000E40090936500809364008091E300909100
:1018F000E40097FF03C091958195910999BD88BD3A
:101900008091E1009091E2002091620030916300AB
:1019100028173907B1F18091E1009091E200892BFD
:1019200019F485B3806C17C08091D000811107C075
:101930008091E1009091E2001816190654F0809110
:10194000D000882351F08091E1009091E20097FF50
:1019500004C085B38F7385BB02C0AE98AF9A8091E7
:10196000E1009091E2009093630080936200809187
:10197000E1009091E20097FF03C091958195910954
:1019800083BD8091DF009091E00020916000309154
:10199000610028173907B1F18091DF009091E000D4
:1019A000892B19F482B38C6017C08091CF0081110C
:1019B00007C08091DF009091E0001816190654F0DE
:1019C0008091CF00882351F08091DF009091E0005A
:1019D00097FF04C082B3837F82BB02C09298939A20
:1019E0008091DF009091E00090936100809360000F
:1019F0008091DF009091E00097FF03C09195819561
:101A000091098CBF8091A9008F5F8093A90085B751
:101A1000806885BF889585B78F7785BF50C96F92DD
:101A20007F929F92AF92BF92CF92DF92EF92FF92FE
:101A30000F931F93CF93DF93CDB7DEB72C970FB6DD
:101A4000F894DEBF0FBECDBF8C017B013A01FC01D3
:101A500017821682838181FF19C1CE0101965C0134
:101A6000F801D380F701D3FC2591D3FE21917F01AA
:101A7000222309F407C1253249F4D3FC2591D3FE72
:101A800021917F01253211F0912C1BC0B801822FCA
:101A900090E00E94941163013601E2CF222309F401
:101AA000F1C0622F70E089E790E02C870E943E1120
:101AB0002C85892B49F0F701D3FC2591D3FE219188
:101AC0007F0197FEEBCF0CC0233221F4F92DF0619A
:101AD0009F2EF1CF2C3639F4292D2068922EEBCF92
:101AE000222309F4CFC0622F70E082E790E02C87B8
:101AF0000E943E112C85892B41F06301F4E0CF0E4A
:101B0000D11CB8018FE390E012C0233641F0233797
:101B100089F0233521F5F92DF1609F2E0BC063016B
:101B200022E0C20ED11CB801F301808191810E9494
:101B30009411B2CF630122E0C20ED11CF301608088
:101B40007180F30190FC859190FE81913F01882383
:101B500009F4A2CFB80190E00E949411F2CF24368C
:101B600011F0293639F5630197FE09C0F4E0CF0E74
:101B7000D11CF30160817181828193810AC0F2E0FE
:101B8000CF0ED11CF30160817181882777FD80958C
:101B9000982FF92DFF7E9F2E97FF09C09095809575
:101BA000709561957F4F8F4F9F4FF0649F2E2AE075
:101BB00030E038C02037A1F040F42835D1F02F367E
:101BC00009F060C028E030E019C0253719F0283747
:101BD00051F058C0292D2F7E922E2AE030E00EC001
:101BE000892D8061982E992D9462992E20E130E004
:101BF00005C0E92DE4609E2E20E132E0630197FEEE
:101C000009C0F4E0CF0ED11CF301608171818281A3
:101C1000938108C0F2E0CF0ED11CF3016081718185
:101C200080E090E0A5010E94F311782E7A1896FECC
:101C300005C0B8018DE290E00E94941194FE16C098
:101C4000FE01E70DF11D8081803381F0B80180E352
:101C500090E00E94941192FE09C0292D2072822FDB
:101C600090E0B801885A9F4F0E9494117A94F50130
:101C7000E70DF11D8081B80190E00E949411711070
:101C8000F5CF0ACFF8018681978102C08FEF9FEFD1
:101C90002C960FB6F894DEBF0FBECDBFDF91CF916B
:101CA0001F910F91FF90EF90DF90CF90BF90AF907A
:101CB0009F907F906F9008955058BB27AA270ED011
:101CC000A0C169D130F06ED120F031F49F3F11F402
:101CD0001EF45EC10EF4E095E7FB54C1E92FB3D1C9
:101CE00080F3BA17620773078407950718F071F439
:101CF0009EF5CBC10EF4E0950B2EBA2FA02D0B0153
:101D0000B90190010C01CA01A0011124FF27591B40
:101D100099F0593F50F4503E68F11A16F040A22F46
:101D2000232F342F4427585FF3CF469537952795B7
:101D3000A795F0405395C9F77EF41F16BA0B620BB6
:101D4000730B840BBAF09150A1F0FF0FBB1F661FFD
:101D5000771F881FC2F70EC0BA0F621F731F841F40
:101D600048F4879577956795B795F7959E3F08F066
:101D7000B3CF9395880F08F09927EE0F9795879525
:101D80000895DCD008F481E0089514D1E3954AC1A8
:101D90000CD037C107D140F0FED030F021F45F3FC6
:101DA00019F0F0C0511172C1F3C04DD198F39923CD
:101DB000C9F35523B1F3951B550BBB27AA2762170F
:101DC0007307840738F09F5F5F4F220F331F441F54
:101DD000AA1FA9F333D00E2E3AF0E0E830D091508C
:101DE0005040E695001CCAF729D0FE2F27D0660F79
:101DF000771F881FBB1F261737074807AB07B0E8B8
:101E000009F0BB0B802DBF01FF2793585F4F2AF0CD
:101E10009E3F510568F0B6C039C15F3FECF3983E74
:101E2000DCF3869577956795B795F7959F5FC9F72A
:101E3000880F911D9695879597F90895E1E0660FB3
:101E4000771F881FBB1F621773078407BA0720F02C
:101E5000621B730B840BBA0BEE1F88F7E095089595
:101E600004D06894B11112C10895F5D088F09F573D
:101E700090F0B92F9927B751A0F0D1F0660F771FD6
:101E8000881F991F1AF0BA95C9F712C0B13081F0B6
:101E9000FCD0B1E00895F9C0672F782F8827B85F8C
:101EA00039F0B93FCCF3869577956795B395D9F717
:101EB0003EF490958095709561957F4F8F4F9F4F21
:101EC0000895E89409C097FB3EF49095809570952D
:101ED00061957F4F8F4F9F4F9923A9F0F92F96E976
:101EE000BB279395F695879577956795B795F111EB
:101EF000F8CFFAF4BB0F11F460FF1BC06F5F7F4F88
:101F00008F4F9F4F16C0882311F096E911C0772399
:101F100021F09EE8872F762F05C0662371F096E8A2
:101F2000862F70E060E02AF09A95660F771F881F71
:101F3000DAF7880F9695879597F90895990F000815
:101F4000550FAA0BE0E8FEEF16161706E807F9078B
:101F5000C0F012161306E407F50798F0621B730B26
:101F6000840B950B39F40A2661F0232B242B252BA7
:101F700021F408950A2609F4A140A6958FEF811D4A
:101F8000811D089597F99F6780E870E060E00895EB
:101F90009FEF80EC089500240A9416161706180681
:101FA0000906089500240A9412161306140605065D
:101FB0000895EECF50D0E8F3E894E0E0BB279F57B8
:101FC000F0F02AED3FE049EC06C0EE0FBB0F661FB4
:101FD000771F881F28F0B23A62077307840728F03A
:101FE000B25A620B730B840BE3959A9572F78038A3
:101FF00030F49A95BB0F661F771F881FD2F7904861
:10200000BAC0092E0394000C11F4882352F0BB0FC0
:1020100040F4BF2B11F460FF04C06F5F7F4F8F4F00
:102020009F4F0895EF93E0FF06C0A2EA2AED3FE03C
:1020300049EC5FEB53DEE5DF0F90039401FC905811
:10204000E4E5F0E0A4C057FD9058440F551F59F047
:102050005F3F71F04795880F97FB991F61F09F3F95
:1020600079F087950895121613061406551FF2CFBE
:102070004695F1DF08C0161617061806991FF1CF0E
:1020800086957105610508940895E894BB27662735
:102090007727CB0197F9089551DF08F48FEF089562
:1020A0000BD0AFCF78DF28F07DDF18F0952309F053
:1020B00069CF6ECF1124EACFC6DFA0F3959FD1F38D
:1020C000950F50E0551F629FF001729FBB27F00DE6
:1020D000B11D639FAA27F00DB11DAA1F649F66273B
:1020E000B00DA11D661F829F2227B00DA11D621F8A
:1020F000739FB00DA11D621F839FA00D611D221F44
:10210000749F3327A00D611D231F849F600D211D27
:10211000822F762F6A2F11249F5750408AF0E1F0CA
:1021200088234AF0EE0FFF1FBB1F661F771F881F13
:1021300091505040A9F79E3F510570F023CFA6CF94
:102140005F3FECF3983EDCF3869577956795B795FE
:10215000F795E7959F5FC1F7FE2B880F911D969528
:10216000879597F908959F9325DF0F9007FCEE5F01
:1021700059CF9F3F31F0915020F48795779567951F
:10218000B795880F911D9695879597F908959F9318
:102190008F937F936F93FF93EF939B01AC0180DF4D
:1021A000EF91FF9105D02F913F914F915F9178CFA3
:1021B000DF93CF931F930F93FF92EF92DF927B01F8
:1021C0008C01689405C0DA2EEF0176DFFE01E894F9
:1021D000A5912591359145915591AEF3EF017EDDA5
:1021E000FE019701A801DA9479F7DF90EF90FF9054
:1021F0000F911F91CF91DF910895052E97FB1EF44B
:1022000000940E94141157FD07D00E941C1107FC76
:1022100003D04EF40C9414115095409530952195AF
:102220003F4F4F4F5F4F0895909580957095619502
:102230007F4F8F4F9F4F0895A1E21A2EAA1BBB1B01
:10224000FD010DC0AA1FBB1FEE1FFF1FA217B30782
:10225000E407F50720F0A21BB30BE40BF50B661F98
:10226000771F881F991F1A9469F76095709580955C
:1022700090959B01AC01BD01CF010895FC01059033
:10228000061621F00020D9F7C00108953197CF013B
:1022900008950F931F93CF93DF93EC018B01009769
:1022A00031F46115710519F480E090E038C06EE0FA
:1022B00070E081E090E00E945112FC010097A1F3D0
:1022C00080E883830115110571F01387028781E887
:1022D000838380915D0190915E01892B21F4F093BD
:1022E0005E01E0935D012097C9F0D187C0878381AB
:1022F0008260838380915F0190916001892B71F4EA
:10230000F0936001E0935F0180916101909162011F
:10231000892B21F4F0936201E0936101CF01DF91F9
:10232000CF911F910F9108950F931F93CF93DF9338
:10233000182F092FEB018B8181FD03C08FEF9FEFD9
:1023400020C082FF10C04E815F812C813D814217E9
:1023500053077CF4E881F9819F012F5F3F4F398358
:102360002883108306C0E885F985812F0995892B7C
:1023700029F72E813F812F5F3F4F3F832E83812F8F
:10238000902FDF91CF911F910F9108950F931F937D
:10239000CF93DF93E0915F01F0916001238121FFF2
:1023A0001BC0EC0100E010E0899160915F01709129
:1023B0006001DB011896ED91FC911997882331F0AB
:1023C0000995892B89F30FEF1FEFEECF8AE009956E
:1023D000892B11F4C80102C08FEF9FEFDF91CF91DD
:1023E0001F910F910895FA01AA27283051F1203149
:1023F00081F1E8946F936E7F6E5F7F4F8F4F9F4F99
:10240000AF4FB1E03ED0B4E03CD0670F781F891FDA
:102410009A1FA11D680F791F8A1F911DA11D6A0FA8
:10242000711D811D911DA11D20D009F468943F915B
:102430002AE0269F11243019305D3193DEF6CF015A
:102440000895462F4770405D4193B3E00FD0C9F720
:10245000F6CF462F4F70405D4A3318F0495D31FD8D
:102460004052419302D0A9F7EACFB4E0A6959795E0
:10247000879577956795BA95C9F7009761057105B6
:1024800008959B01AC010A2E069457954795379500
:102490002795BA95C9F7620F731F841F951FA01D5A
:1024A00008950F931F93CF93DF93869F8001879F9B
:1024B000100D969F100D1124C8010E946D12EC01A1
:1024C000009729F0A80160E070E00E949413CE010B
:1024D000DF91CF911F910F910895CF93DF938230B9
:1024E000910510F482E090E0E0916501F0916601C1
:1024F00020E030E0A0E0B0E0309739F14081518138
:1025000048175907B8F04817590771F48281938129
:10251000109729F013969C938E9312972CC090934A
:1025200066018093650127C02115310531F04217FE
:10253000530718F0A901DB0101C0EF019A01BD01A9
:10254000DF010280F381E02DD7CF21153105F9F0AD
:10255000281B390B2430310580F48A819B81611559
:10256000710521F0FB019383828304C0909366017F
:1025700080936501FE01329644C0FE01E20FF31F15
:102580008193919322503109398328833AC0209155
:10259000630130916401232B41F420916A00309152
:1025A0006B003093640120936301209168003091A7
:1025B00069002115310541F42DB73EB740916C00FB
:1025C00050916D00241B350BE0916301F091640183
:1025D000E217F307A0F42E1B3F0B2817390778F0FA
:1025E000AC014E5F5F4F2417350748F04E0F5F1F59
:1025F00050936401409363018193919302C0E0E0A2
:10260000F0E0CF01DF91CF910895CF93DF93009752
:1026100009F487C0FC01329713821282C0916501D0
:10262000D0916601209781F420813181280F391FD4
:1026300080916301909164018217930779F5F0937B
:102640006401E09363016DC0DE0120E030E0AE176D
:10265000BF0750F412964D915C9113979D0141155F
:10266000510509F1DA01F3CFB383A283408151818F
:10267000840F951F8A179B0771F48D919C91119778
:10268000840F951F02969183808312968D919C9161
:102690001397938382832115310529F4F093660102
:1026A000E09365013EC0D9011396FC93EE93129717
:1026B0004D915D91A40FB51FEA17FB0779F4808156
:1026C0009181840F951F0296D90111969C938E9348
:1026D0008281938113969C938E931297E0E0F0E0B1
:1026E0008A819B81009719F0FE01EC01F9CFCE01A0
:1026F000029628813981820F931F209163013091C6
:1027000064012817390769F4309729F4109266019B
:102710001092650102C013821282D0936401C093AB
:102720006301DF91CF910895DC0101C06D934150A9
:0A2730005040E0F70895F894FFCF41
:10273A0000800080008000800000670120000D0AF0
:08274A0053746172740D00006C
:00000001FF
